:0200000480007A
:100000009710000093800000171100001301810178
:1000100083A1000013020000930210001303F0FFFD
:10002000B70300809383F3FF37040080930F000031
:100030006394410093EF1F006394510093EF2F00EE
:100040006394610093EF4F006394710093EF8F000E
:100050006394810093EF0F0123203100232241009C
:10006000232451002326610023287100232A8100C4
:10007000232CF10197100000938000F91711000064
:10008000130101FC03A300009303000013041000FC
:100090009304F0FF370500801305F5FFB7050080D6
:1000A000930F00006314730093EF1F006314830029
:1000B00093EF2F006314930093EF4F006314A3009A
:1000C00093EF8F006314B30093EF0F0123206100BF
:1000D0002322710023248100232691002328A100DC
:1000E000232AB100232CF10197100000938000F225
:1000F00017110000130181F603A60000930600000B
:10010000130710009307F0FF370800801308F8FF6B
:10011000B7080080930F00006314D60093EF1F0010
:100120006314E60093EF2F006314F60093EF4F0083
:100130006314060193EF8F006314160193EF0F0110
:100140002320C1002322D1002324E1002326F10033
:1001500023280101232A1101232CF101971000000B
:10016000938000EB17110000130101F103A90000B7
:1001700093090000130A1000930AF0FF370B008068
:10018000130BFBFFB70B0080930F000063143901C2
:1001900093EF1F006314490193EF2F00631459017B
:1001A00093EF4F006314690193EF8F00631479019B
:1001B00093EF0F0123202101232231012324410148
:1001C0002326510123286101232A7101232CF101E7
:1001D00097100000938000E417110000130181EBD9
:1001E00003AC0000930C0000130D1000930DF0FF02
:1001F000370E0080130EFEFFB70E0080930F000035
:1002000063149C0193EF1F006314AC0193EF2F0064
:100210006314BC0193EF4F006314CC0193EF8F0084
:100220006314DC0193EF0F0123208101232291014C
:100230002324A1012326B1012328C101232AD101AE
:10024000232CF101971D0000938D8DE69300000093
:10025000130110009301F0FF370200801302F2FF38
:10026000B7020080930F00006394000093EF1F001B
:100270006314010093EF2F006394010093EF4F008C
:100280006314020093EF8F006394020093EF0F0159
:100290006314100093EF0F026314200093EF0F0418
:1002A0006314300093EF0F086314400093EF0F10B6
:1002B0006314500093EF0F2023A0FD01971A000054
:1002C000938A8AD5171B0000130BCBDE83AF0A007D
:1002D0001301F0FF9301F0FF37D2ED0F130292BA32
:1002E00063940F0213010000930100001302000049
:1002F000B74165879381113263940F0213010000A7
:10030000930100001302000037E1BC9A130101EFD2
:10031000E3900FFE130100009301000013020000A0
:1003200023200B0023222B0023243B0023264B00F9
:1003300017150000130505CF97150000938585D884
:10034000370610F01306C6F26306B5028326C50011
:100350002320D600832685002320D600832645004F
:100360002320D600832605002320D600130505018F
:100370006FF09FFD370510F0130505F223200500EF
:040380000000000079
:101000000000000001000000FFFFFFFFFFFFFF7F67
:1010100000000080FFFFFFFF000000000000000054
:10102000FFFFFFFFFFFFFFFFFFFFFFFFFFFFFFFFD0
:10103000FFFFFFFFFFFFFFFFFFFFFFFFFFFFFFFFC0
:10104000FFFFFFFFFFFFFFFFFFFFFFFFFFFFFFFFB0
:10105000FFFFFFFFFFFFFFFFFFFFFFFFFFFFFFFFA0
:10106000FFFFFFFFFFFFFFFFFFFFFFFFFFFFFFFF90
:10107000FFFFFFFFFFFFFFFFFFFFFFFFFFFFFFFF80
:10108000FFFFFFFFFFFFFFFFFFFFFFFFFFFFFFFF70
:10109000FFFFFFFFFFFFFFFFFFFFFFFFFFFFFFFF60
:1010A000FFFFFFFFFFFFFFFFFFFFFFFFFFFFFFFF50
:1010B000FFFFFFFFFFFFFFFFFFFFFFFFFFFFFFFF40
:040000058000000077
:00000001FF
